:020000040000FA
:0600000000000EEF00F00D
:0400080027EF00F0EE
:0800180028EF00F001D8FFD72A
:10002000480E046EE80E056E010E066ED00E946E3C
:10003000810ECD6E080EBD6ED08E9F909F94026A89
:10004000020E036E9D849D80F28CF28E12001100D0
:10005000D8CF01F0006E9EA402D00BD8FCD79EA092
:1000600002D019D8F8D701D0F6D7005001C0D8FF78
:1000700010009EA004D0BFBE02D0022A9E90025063
:10008000035C07E1BD700450BE260550BF22065038
:0C00900003229E941200022A9E9012008F
:020000040030CA
:08000000FFFAF6FEFFFFFBFF13
:00000001FF
